:020000020000FC
:0200000001C33A
:0200040018954D
:02000800189549
:02000C00189545
:02001000189541
:02001C00189535
:0200240018952D
:0200280085C091
:02002C00A3C06F
:02003000189521
:02004000189511
:020044005EC09C
:02004800189509
:02004C00189505
:02005000189501
:020054001895FD
:020058001895F9
:02005C001895F5
:020060001895F1
:020064001895ED
:020068001895E9
:02006C001FC0B3
:020070001895E1
:020074001895DD
:020078001895D9
:02007C001895D5
:020080001895D1
:020084001895CD
:020088001895C9
:02008C001895C5
:020090001895C1
:020094001895BD
:020098001895B9
:02009C001895B5
:0200A0001895B1
:0200A4001895AD
:0200A8001895A9
:1000AC002FB6DF2DCE2DD63039F418607091C900E3
:1000BC007F7B7093C9001DC00E94880E7991FD2E24
:1000CC00EC2EF09914C0D0912F01D03881F00F9202
:1000DC001F92D79F17FE02C07FEF05C0712D70389D
:1000EC0010F07FEF02C0000C771F1F900F907093E1
:1000FC00CE002FBE18952FB60260DD2009F0DA94E1
:10010C00CA9409F010C07AE0C72E0460F09B06C0B8
:10011C0000005D9B02C05D9801C05D9ABA9409F025
:10012C0002C0B72E0160E5CF2FB67091E10073FFCE
:10013C0019C07091E100777E7093E100772770937E
:10014C00E9007091EB0071607093EB0070E07093BC
:10015C00EC0070E072607093ED007091F0007860CC
:10016C007093F0002FBE18952FB68F937091F400FA
:10017C0070FF07C070E07093E9007091E80073FDA8
:10018C000DD07091F40072FDD6D1F79B04C0709124
:10019C00F40073FD13D28F912FBE1895EF93FF933C
:1001AC007091F100709305017091F100709306014C
:1001BC007091F100709308017091F1007093090136
:1001CC007091F10070930A017091F10070930B0122
:1001DC007091F10070930C017091F10070930D010E
:1001EC007091E800777F7093E80070910501F79BA0
:1001FC0006C0713209F47DC0713A09F470C0717691
:10020C0019F0713009F00BC070910601703041F09B
:10021C007530A9F0763039F1793009F485C0E0C039
:10022C0077277093F1007093F1007091E8007E7F56
:10023C007093E8007091E80072FFFCCFD6C070910B
:10024C0008017F777093E3007091E8007E7F7093D4
:10025C00E8007091E80070FFFCCF7091E3007068CB
:10026C007093E300C2C070910901713029F07230B3
:10027C0069F0733021F1B4C0F79B03C0EEE1F2E2F8
:10028C0002C0ECEEF2E2D491B3D0AFC0D0910C012D
:10029C00D03049F070910D01703029F4F79BD536B0
:1002AC00F799D33420F0F79BD5E6F799D3E4F79B75
:1002BC0003C0E0E7F2E211C0EAEFF2E20EC0709187
:1002CC000801772319F4E4EBF2E206C0713019F45B
:1002DC00E6ECF2E201C084C0D491F6D086C07091F5
:1002EC000601713209F07CC0E2EEF2E2D7E0ECD00C
:1002FC007CC070910601703251F47091E80072FF6D
:10030C00FCCF7091E8007B7F7093E80003C07232E1
:10031C0009F066C07091E8007E7F7093E8007091E0
:10032C00E80070FFFCCF61C0F79BC2E0F799C3E017
:10033C00C093E9007091EB007E7F7093EB0070919D
:10034C00ED007D7F7093ED00CA9591F771E070938D
:10035C00E9007091EB0071607093EB0071E87093A1
:10036C00EC0070E372607093ED0077277093F000EF
:10037C0072E07093E9007091EB0071607093EB0088
:10038C0070E87093EC0070E372607093ED00709104
:10039C00F00074647093F000F79B14C073E07093DA
:1003AC00E9007091EB0071607093EB0071EC70934D
:1003BC00EC0070E172607093ED007091F000716070
:1003CC007093F00077277093E9007091E8007E7FBE
:1003DC007093E8007091E8007170E1F3F69A05C033
:1003EC007091EB0070627093EB00FF91EF910895A8
:1003FC0070910D01772331F470910C017D1708F485
:10040C00D72FCC277091E80072FD94C07591709332
:10041C00F100DA95C395C830A9F77091E8007E7F9A
:10042C007093E8007091E8007570E1F37091E8004A
:10043C0072FD80C0EF93FF938F939F935F9355272B
:10044C00F1E0E8E00E94560B802D0E94560B902D97
:10045C00813411F4933211F0982B41F481E48093A0
:10046C00F10083E28093F1005FEF04C08093F10010
:10047C000092F1000E94560B802D0E94560B902D7D
:10048C00863321F4903011F4552321F40E94560B3D
:10049C00002061F486E390E0F79B92E80000F79B64
:1004AC0086E38093F1009093F10006C0F79B0196D0
:1004BC008093F1009093F1005F919F918F91FF9148
:1004CC00EF91CCE0D45014C070910D01772329F436
:1004DC0070910C017D1708F4D72FCC277091E80090
:1004EC0072FD28C0A89575917093F100DA95C395AB
:1004FC0077E07C2349F47091E8007E7F7093E800EC
:10050C007091E8007570E1F3D03041F77091E8001C
:10051C00747009F00AC07091E8007E7F7093E80057
:10052C00A8957091E80072FFFBCF7091E8007B7F7B
:10053C007093E80008955F9372E07093E9007091F6
:10054C00E80072FF39C07091E8007B7F7093E8007F
:10055C0010FD32C07091F200772309F1D62DC72D12
:10056C005091F1005993D53011F4D2E0C0E06D2ECA
:10057C007C2E6F93572D662D681430F009F005C052
:10058C00791410F049F001C06D5F59196809623097
:10059C0018F05F3B08F011606F917A9509F710FD28
:1005AC000BC07091E8007B7F7093E80000007091A5
:1005BC00E8007F777093E8005F9108955F9373E094
:1005CC007093E9007091E80070FF14C0707A70931A
:1005DC00E80011FF09C0C0ECD1E070910F015991F6
:1005EC005093F1007A95D9F71D7F7091E8007F77D1
:1005FC007093E8005F910895F89491E09EBF9CEF92
:10060C009DBF88279FEF84B995B987B998B98AB9E6
:10061C009BB98DB99EB980BB91BB002711272227AE
:10062C00CC24C394BC2CF1E0E0E099279193F130F9
:10063C00E8F3539A5B9A379907C0F1E0E8E0552745
:10064C000E94610BED30D9F7519A59980E94D50C44
:10065C009927909380009CE09093810092E081E731
:10066C00909389008093880092E090936F0090B7EC
:10067C00906890BF8EE19EE0809360009093600044
:10068C0099279EBB0E944A0B90931B010E948D0BD5
:10069C000E94700BA895F69BFDCF0E94780B0E94D0
:1006AC004A0B90931B01559A209A28985D98F1E07B
:1006BC00E4E00E94560B00922301A895A8954427CC
:1006CC00332718600E94D50C0E942F0C0E94500AF0
:1006DC000E944A0EF79905C02ED7F6F70E948C0E91
:1006EC00FBCF29D7F6F7F3D0FCCF6F938F939F9363
:1006FC00982F6091110163956093110197FF50C081
:10070C00903F29F42160217F90931201DCC0973F28
:10071C0019F56130A9F1623081F097E090931001E6
:10072C0090911301909312019091140190931301E5
:10073C0097EF90931401207F95C096E09093100151
:10074C00909113019093120197EF909313019927B5
:10075C0090931401207F86C090931201943FE8F08F
:10076C00983F89F09E3F79F09A3F69F09B3F59F092
:10077C009C3F49F09F3F39F0963F29F0247F9FC062
:10078C0097EF909312019927909313019093140172
:10079C0095E090931001207F65C02160217F93C06C
:1007AC0020FD0CC0207F909312019FE090931001CC
:1007BC009927909313019093140154C021FD1EC0EE
:1007CC009093130199279093140190911201913FEA
:1007DC0079F0933F69F0907F903C21F0903D11F0BF
:1007EC00226071C09295909310012160217F3AC0D4
:1007FC0092E0909310012160217F34C020FF5FC0F4
:10080C0022FD18C09093140123FF02C024605BC02A
:10081C0090911201923F49F0903FF9F092959F70A0
:10082C00909310012160217F1DC093E090931001E3
:10083C00207F18C020FF43C022FF41C080911301CC
:10084C0080931201809114018093130190931401F1
:10085C0094E090931001297F05C094E090931001CF
:10086C00297F2860F894000091E09093E900A89506
:10087C009091E80090FFFBCF9E7B9093E8009091C5
:10088C0010019093F100909112019093F1009091CE
:10089C0013019093F100909114019093F1009091B9
:1008AC00E8009E7F9093E80000009091E8009F770D
:1008BC009093E800789499279093110104C099279C
:1008CC0090931101207F9F918F916F910895F09BD0
:1008DC0005C0A8959A3509F008958BC0923011F097
:1008EC00933019F40E943A06A3C09A3519F4D6D065
:1008FC001F789EC0F0999CC0963511F4F0D198C029
:10090C00933511F4D6D194C0943508F064C090346A
:10091C0008F026C0933219F40E94660689C09432FE
:10092C0019F40E944A3F84C0963219F40E94483F41
:10093C007FC09B3219F40E94CD0B7AC09C3211F40B
:10094C00C8D176C09D3219F40E94E20B71C09D3360
:10095C0011F4CDD16DC09F3319F40E94A60868C064
:10096C00903419F40E942B0C63C0913411F450D2C2
:10097C005FC0923411F405D25BC0933419F40E9419
:10098C00F40556C0943419F40E94A70C51C0973446
:10099C0019F40E9401074CC0983419F40E94B30654
:1009AC0047C09D3411F4F6D143C09E3439F4909174
:1009BC003B01923010F00E942E073AC0903511F492
:1009CC003DD236C0913519F40E947B0731C0923567
:1009DC0011F461D22DC0943511F463D329C097352D
:1009EC0019F40E94BC0624C0983519F40E946C3F7F
:1009FC001FC0953511F4B0D01BC09E3519F40E9460
:100A0C004C3F16C09F3519F40E945F3F11C09C37B4
:100A1C0019F40E94C00C0CC09E3719F40E94EE0B06
:100A2C0007C09D3009F435C09A3011F0903209F4AA
:100A3C000895F79909C080912301806C0E947B0373
:100A4C008FE30E947B0305C08FE30E94FD0A0E9486
:100A5C00FC0A40D692E0692E892E90E0792E992ED0
:100A6C00F8940000E2E0E093E900E091E800EB7F0D
:100A7C00E093E8000000E091E800EF77E093E800F5
:100A8C001E78F098077E91E09EBF9CEF9DBF7894F6
:100A9C0021CEF79B08950E94FC0A08959AE0D92E66
:100AAC00A89549D5DD2019F4F09BC3CF0895CEF756
:100ABC009A35A1F31F79913A81F01064923A69F05A
:100ACC009AE0D92EA895DD2039F035D5E6F79A3580
:100ADC0029F3953A09F0F7CF27C008601061F09A16
:100AEC00AA27A0933B01A0933C01A0933E01BB27F6
:100AFC00F7E0E0E096E0D92EDD20B1F01CD5E6F76A
:100B0C00F93008F491931196BB23A1F3B23011F094
:100B1C0015FDF0CFA13071F716FF04C015FD02C012
:100B2C001062E8CF953A41F08AE561D581EC5FD54A
:100B3C0085EA5DD5077F0895F7E0E0E0B5E0A0E039
:100B4C0091919D93B630E1F78AE551D581EC4FD563
:100B5C0085EA4DD5077F08953F925F936F930F936E
:100B6C000062F198F2989FE786EE0E943F0B98D0B6
:100B7C0066F4332E832FF19A5AD5F19891D02EF436
:100B8C00832FF19A54D5F19801C026C0532F9FE7BB
:100B9C008CEE0E943F0B84D06EF4832FF19A0E944E
:100BAC001D0BF198432E7CD02EF4832FF19A3FD558
:100BBC00F19801C011C0F1E0E8E07DD5532D7BD553
:100BCC00532F79D5542D77D55AE575D5B9D20F91C8
:100BDC006F915F913F9008950C941F059FE78EECE9
:100BEC0048D58AE304D582E020D30EF03BC00F7EBB
:100BFC003A3010F4832F04C081E3F9D4832F8A5048
:100C0C00805D0E94FD0A532F552361F1513150F53F
:100C1C005F939FE78CED2DD59FE78EEC2AD58AE369
:100C2C00E6D482E002D35F910EF01CC00F7E3A3006
:100C3C0010F4832F04C081E3DAD4832F8A50805DB3
:100C4C000E94FD0A0F7E351769F480E2D0D48FE63E
:100C5C00CED48BE6CCD48DE0CAD4F1E0E4E05A9546
:100C6C002AD508950C941F0508609170F92F0E94E5
:100C7C00A10AEEF7E92F9F2B09F4F2E00E94B60BC4
:100C8C000E94A10AEEF7077F092E309127014091AF
:100C9C0028010E94CE0D309327014093280108951E
:100CAC0082E0FCD226F4442311F468940895E8946D
:100CBC00089583E00E941B0916F40E94B10D08955B
:100CCC0083E00E941B0926F40E94B10D0E94C80DFE
:100CDC0008950E940C0956F40E94B90B03C00E949F
:100CEC000C0926F430932A010E94C80D089583E064
:100CFC000E941B090EF00895442371F58091270181
:100D0C00909128018F3F08F027C08F939F93E82F75
:100D1C00F92FFE5F008000922A0101968093270133
:100D2C0090932801332389F03F938F939F930E94D4
:100D3C00C80D9F918F913F910196803031F0809337
:100D4C002701909328013A9569F79F919093280178
:100D5C009F919093270108956CCE0E940C090EF080
:100D6C000895309331010E940B0D08950E940C09D7
:100D7C000EF0089530953695309333010E940B0D8B
:100D8C0008950E940C090EF00895309332010E94D0
:100D9C000B0D089583E00E941B090EF00895393C59
:100DAC0008F047CE30933001343611F430E820C0CF
:100DBC00393B10F096E015C0363910F095E011C0B3
:100DCC00383710F094E00DC0353510F093E009C0C1
:100DDC00323310F092E005C03F3010F091E001C0CA
:100DEC009927532F56955695350F390F08F43FEF29
:100DFC0030932F01089583E00E941B090EF0089593
:100E0C00442329F43A3518F430933A0110C011CE2A
:100E1C0083E00E941B090EF008954423C1F73A3574
:100E2C00B0F73130A1F330933B01332309F031E0BB
:100E3C0030933E01332730933C01089583E00E94A8
:100E4C001B090EF0089530933D0130933E01089537
:100E5C003F934F93EF93FF9380913D0180933E011D
:100E6C0080913C019927442730913A01380F3A354B
:100E7C0008F033270E94770CFF91EF914F913F912F
:100E8C0080913C01839590913B01891709F4882747
:100E9C0080933C01089583E00E941B090EF0089595
:100EAC00442309F021C0313808F030E883E70E9470
:100EBC00FD0A90912601809125010E94A30986E7E5
:100ECC000E94FD0AF5E0E0912501EA9581910E94CE
:100EDC009209E03031F03A9521F08CE20E94FD0A43
:100EEC00F5CF0E94FC0A0895A4CD0F921F9283E4C3
:100EFC000E94FD0A88E40E94FD0A8DE30E94FD0A0F
:100F0C0080912501682F909126010E94A30980E20F
:100F1C000E94FD0AF0912801E0912701FE5F5081AB
:100F2C0086E40E94FD0A89E60E94FD0A8EE60E9474
:100F3C00FD0A8DE30E94FD0A852F0E94920980E232
:100F4C000E94FD0AF0912801E09127016E2F51912A
:100F5C005F9384E50E94FD0A88E50E94FD0A8DE3FB
:100F6C000E94FD0A852F0E94920980E20E94FD0AD0
:100F7C0082E50E94FD0A8DE30E94FD0A5F91852F98
:100F8C0090912F01903841F0899F812D803810F07D
:100F9C008FEF02C0000C881F0E94920980E20E9411
:100FAC00FD0A6F3F91F187E40E94FD0A8DE30E94D8
:100FBC00FD0A819190912F01903841F0899F812DEC
:100FCC00803810F08FEF02C0000C881F0E9492092D
:100FDC0080E20E94FD0A6E3FC1F082E40E94FD0A8D
:100FEC008DE30E94FD0A808190912F01903841F091
:100FFC00899F812D803810F08FEF02C0000C881F64
:10100C000E94920980E20E94FD0A0F938DE40E94D7
:10101C00FD0A86E40E94FD0A8DE30E94FD0A0F7B07
:10102C00809130010E94050A85E20E94FD0A80E24F
:10103C000E94FD0A83E40E94FD0A83E50E94FD0ADA
:10104C008DE30E94FD0A80913A010E94050A8FE20D
:10105C000E94FD0A80913B010E94050A8FE20E94CA
:10106C00FD0A80913D018F770E94050A80E20E9463
:10107C00FD0A84E50E94FD0A8DE30E94FD0A809121
:10108C002B010E94050A8EE20E94FD0A80912C0120
:10109C000E94050A0F918DE00E94FD0A1F900F908F
:1010AC000895992790932B0190932C0183E0BDD048
:1010BC000EF0BFCC423008F0BCCC5F93552799277B
:1010CC00442311F099E156E0332361F03A3018F0E3
:1010DC003A509395FBCF350F3A3010F03A50939528
:1010EC005F9102C0352F5F91903210F09FE139E093
:1010FC0090932B013A3008F039E030932C01002406
:10110C004427990F892F990F990F890F041E890F66
:10111C00041E890F041E890F041E890F041E890FDB
:10112C00041E880F001C330F432F330F330F340F63
:10113C004427830F041E00922D0180932E010895E5
:10114C009EE78CEE0E943F0B9FE784E20E943F0BD0
:10115C009FE786EE0E943F0BF1E0E8E00E94560B01
:10116C00902D0E94560B802D892B11F0802D02C0E2
:10117C0091E483E20F930062F19A59D2F198892F8E
:10118C0056D29FE78CEE0E943F0BF1E0EAE00E9402
:10119C00560B802D0E94560B502D0E94560B002092
:1011AC0011F0952F02C086E390E0F79902C092E807
:1011BC0086E3582F892FF19A3AD2F198852F37D29E
:1011CC0080E215D214D29FE78EEC0E943F0B8DE388
:1011DC000ED2F1E0E4E00E94560B00922301902D18
:1011EC0093959A3010F4892F04C081E300D2892F93
:1011FC008A50805D0E94FD0A8DE0F9D19FE78EE355
:10120C000E943F0B0F9108950C941F0506FF04C01C
:10121C0082E044D03EF403C083E007D01EF44423A4
:10122C0011F4689408950C941F0585D1F6F73327B3
:10123C0044278F9302C07FD1F6F79D3039F19A3055
:10124C0029F1903278F0B9F39C32A9F39E3299F3DC
:10125C009033E0F09734D0F4913420F49A33B0F416
:10126C0052D016F00C941F05330F441F532F642FCC
:10127C00330F441F330F441F350F461F6627390F9A
:10128C00461F8A95C1F668948F91089500619F91CD
:10129C00891711F4E8940895689408958F9333276F
:1012AC00442749D1F6F79D3089F3973F11F49DE01F
:1012BC00EDCF9032E8F0A9F3903340F3973430F748
:1012CC00913410F49A3310F718D016F00C941F05C3
:1012DC00330F441F330F441F330F441F330F441F6E
:1012EC006627390F461F8A95E1F668948F91089509
:1012FC000C941F05913470F002C0913420F0973497
:10130C0048F4975305C0903328F090539A3010F45A
:10131C0068940895E89408959F93992706FF0AC04E
:10132C008F9384E2F79963D10000F79BDED98F91FC
:10133C0066D001C064D09F9108950F930F7D5F9389
:10134C006F933F92582F992369F19732B0F011F4B3
:10135C00503198F087E2382E60E18827931540F0E1
:10136C0011F4561728F083950062561B9309F6CF9B
:10137C008063F7993CD1F79BB8D983E0382E68EE9F
:10138C008827931540F011F4561728F083950062C6
:10139C00561B9309F6CF806305FF04C0F79927D13C
:1013AC00F79BA3D98827332464E6992311F45617A5
:1013BC0028F083950062561B9309F7CF806305FFD5
:1013CC0004C0F79914D1F79B90D988276AE0561777
:1013DC0020F083950062561BFACF806305FF04C092
:1013EC00F79905D1F79B81D9852F8063F799FFD0A9
:1013FC00F79B7BD93F906F915F910F9108950F935D
:10140C0006FF1BC09F93982F82958F7005FD41F0AE
:10141C00805D8A3308F0895FF799E9D0F79B65D92D
:10142C00892F8F70805D8A3308F0895FF799DFD040
:10143C00F79B5BD99F910F9108959F935F93982F82
:10144C008827943660F054E680E38395951B943698
:10145C00E0F79F93F799CBD0F79B47D99F918823BF
:10146C0011F49A3068F05AE080E39A3018F08395C2
:10147C00951BFBCF9F93F799BAD0F79B36D99F91C9
:10148C00892F805DF799B3D0F79B2FD95F919F91EE
:10149C000F910895A89501FF4AC00D7F992790934D
:1014AC003701F09918C012FD0E94180E02FF13C0EC
:1014BC000B7F90913B01992371F080913D01882322
:1014CC0051F080913E01882331F08A9580933E0142
:1014DC0011F40E942E0700FF21C00E7F14FD05C0E1
:1014EC000000F09B02C0F0985D98CED080911B015B
:1014FC008917A1F05D9A99279093D800A8950000C0
:10150C00FECFF8940E94700B81E08EBF8CEF8DBFE4
:10151C007894A8950E94780B0C9455038091150132
:10152C00882329F08A958093150109F45D9813FDA1
:10153C000E94590E08958F93EF93FF93ABDF04FF36
:10154C0004C0909138010F7E3CC0E894F82DE92D31
:10155C00972D9E1721F4962D9F1709F443C0919156
:10156C00F53011F4F2E0E0E08F2E9E2E5F936F9336
:10157C00572D662D681430F009F005C0791410F061
:10158C00E1F001C06D5F59196809623010F0503BF1
:10159C00A0F410FF12C01E7FF8940000F2E0F0934C
:1015AC00E900F091E800FB7FF093E8000000F09177
:1015BC00E800FF77F093E80078946F915F91909337
:1015CC003801F79B07C003FD05C09B3718F4913613
:1015DC0008F090520F7E6894F09904C0E9E1E09312
:1015EC0015015D9AFF91EF918F9108958DE08F9386
:1015FC00F894000081E08093E900A8958091E800C0
:10160C0080FFFBCF8E7B8093E8008F918F9380932C
:10161C00F1008091E8008E7F8093E80000008091BB
:10162C00E8008F778093E80078948F9108958F93DA
:10163C0005FD02C080E2DBDF8F918F9382958F7066
:10164C00805D8A3308F0895FF19908C0F29B02C073
:10165C00803329F0803311F4F19B80E2C8DF8F9145
:10166C008F938F70805D8A3308F0895FC0DF8F9114
:10167C000895FF93EF93FC018591882311F0B7DF58
:10168C00FBCFEF91FF9108951D9B05C09927F79A09
:10169C00F498F39804C09FEFF798F49AF398089590
:1016AC0003D0009431960895F2BDE1BD002403945B
:1016BC000FBA00B40895509502D031960895A895AC
:1016CC00F894F2BDE1BD50BDFA9AF99AF999FECFA2
:1016DC00789408959F939AEFA8950AD09A95E1F77C
:1016EC009F910895F7DFF6DFF5DFF4DFF3DF089560
:1016FC009F9398EC992349F09F939F919F939F916F
:10170C000000000000009A95F5CF9F9108950024E9
:10171C0091E09093D70090EB9093D80000009F7DC0
:10172C009093D800000090629093D80090E199BDFE
:10173C00926099BD99B590FFFDCF9091D8009F7D97
:10174C009093D80099279093E00098E09093E20052
:10175C0092E0692E892E90E0792E992E7894089536
:10176C00FB5F31970895E0912501F0912601FF234D
:10177C0061F43196E0932501F09326010E94B60B9B
:10178C00F0932801E093270108950C941F05F09124
:10179C002801E09127015081FE5F0080902D9F3F32
:1017AC0049F00394008200922A01F250951719F423
:1017BC00008201C0F2500895F0912801E0912701B8
:1017CC005081FE5F0080902D9923A1F30A94EACFFB
:1017DC0082E00E941B09C6F53A3510F00C941F05E7
:1017EC0013FFFECFAF93BF93EF93FF933F93F4E2BE
:1017FC00F30FEE27A0E0B7E09BE5909337010E9432
:10180C00023FE0E89BE5909337010E94023F992745
:10181C00909337013F91332399F4F1E0E0E050913C
:10182C002D010E94610B50912E010E94610B5FEF04
:10183C0006FD55270E94650B3196522F0E94610BB5
:10184C00FF91EF91BF91AF91089582E00E941B0927
:10185C00DEF73A3510F00C941F053323B1F4F1E0A8
:10186C00E0E00E94560B00922E010E94560B009253
:10187C002D010E945A0B0F7B01FE006431960E94D1
:10188C00560B902D907F2F70292BAF93BF93EF9316
:10189C00FF93F4E2F30FEE27A0E0B7E0A8950590D4
:1018AC0000940D92A030D9F7F5E0E0E0B7E0A0E0AD
:1018BC00A8950C905081501559F080912E01909163
:1018CC002D01992321F4882311F4008201C07AD1CF
:1018DC0031961196F63061F7FF91EF91BF91AF9170
:1018EC0008953A3510F00C941F05AF93BF93EF9306
:1018FC00FF93F4E2F30FEE27A0E0B7E0A895059074
:10190C0000940D92A138D9F7F5E0E0E0B7E0A0E043
:10191C00A8950C905081501559F080912E01909102
:10192C002D01992321F4882311F4008201C04AD19E
:10193C0031961196E13861F7FF91EF91BF91AF911C
:10194C0008959FE78CED95DE0E94A10AEEF79F7D2E
:10195C00943411F00C941F058DE049DEF894F5E0F9
:10196C00E0E0B7E0A0E0992791939D93F630E1F782
:10197C00789408959FE78CED7CDE0E94A10AEEF727
:10198C009C3711F00C941F05F894F1E0E4E0552716
:10199C0092DEA8DEA7DEA6DE8DE00E94FD0AF8949A
:1019AC00F5E0E0E099279193FB30E9F70F7B1F7B83
:1019BC00992790932A0190932B0190932C0190934B
:1019CC002D0190932E019093260182E380933A018E
:1019DC0090933B019093390184E180933D01939561
:1019EC0090932501909333019FEF9093320190E8EF
:1019FC0090932F0194E69093300195E090932801F9
:101A0C0090E09093270178940895309131013B3206
:101A1C0038F4330F5FEF531B330F632F882742C00B
:101A2C00353580F43B52432F4695469546956BEAE7
:101A3C00330F630F330F339533955CEA531B541BF1
:101A4C00882730C0303840F43555330F6FEF631BA7
:101A5C00330F832F552726C03A3A80F43058432F42
:101A6C004695469546958BEA330F830F330F339586
:101A7C0033956CEA631B641B552714C0353D40F449
:101A8C003A5A330F8FEF831B330F532F66270AC03D
:101A9C00355D5BEA330F530F330F339533958AEA79
:101AAC00831B66271F92909133019F779923C1F076
:101ABC009F3709F490E84FEF451B499F412D000CCF
:101ACC00441F540F4FEF461B499F412D000C441FE0
:101ADC00640F4FEF481B499F412D000C441F840F8E
:101AEC00909132019F3F69F09695599F512D000CB2
:101AFC00551F699F612D000C661F899F812D000C5D
:101B0C00881F1F9060933501809336013091250119
:101B1C004091260150932A010E94C80D0090350176
:101B2C0000922A010E94B90B0E94C80D0090360148
:101B3C0000922A010E94B90B0E94C80D3093250116
:101B4C0040932601E32FF42F0E94B60BF09328014B
:101B5C00E09327010895442329F0423088F433237D
:101B6C0079F402C0332361F03093250140932601B0
:101B7C00E32FF42FF5DDF0932801E093270108956E
:101B8C000C941F05F0912801E091270100902A0187
:101B9C0000922A01F0932801E093270150815015FF
:101BAC0009F40EC0FE5F0082F25080912E019091DC
:101BBC002D01992321F4882311F4008201C002D055
:101BCC0078940895501908F45195002480912E01B1
:101BDC0090912D010AD0FD5F9083F3958083882727
:101BEC00F3958083F550146008954F923324441874
:101BFC0061E1001C551F6A9551F4969587958319E0
:101C0C009409802D952F08F401964F900895331C5C
:101C1C00441C381A490A20F4380E491E8894E9CF1E
:101C2C000894E7CF5F936F933F92F5E0E0E01B7F62
:101C3C008081FE5F9081891711F4F2501DC0F395DD
:101C4C005081F3956081F3953080360E08F45395EE
:101C5C003082891740F4850F20F0981710F014602B
:101C6C0009C0892F07C0851B20F0891710F014605C
:101C7C0001C0892FF55080833196E03009F0D8CF20
:101C8C003F906F915F910895599A93E09093CC0097
:101C9C009091C8009D7F9093C80099279093C9009C
:101CAC009EE09093CA000E947E0BF8949091C9001C
:101CBC00977B9093C9005B98539A78940E947E0B03
:101CCC005B9A14D01FD0F89495E0F92EEE249091E5
:101CDC00C90098649093C90099279093CE00177F00
:101CEC00789408959F9392E00C94800B9F9390E1CD
:101CFC000C94800B9F9390EB0C94800B9F9390E033
:101D0C000C94800B9F9394E00C94800B892F8F7014
:101D1C008F3011F0883050F40E94A10AEEF70E9427
:101D2C00A10AEEF70E94A10AEEF70895892F907F81
:101D3C0099F70E94A10AEEF790932001FCDBF6F7CD
:101D4C0090932101F8DBF6F79093220190912001FA
:101D5C00907F903A61F0903D51F0909120019F70EE
:101D6C0080912301981B29F010F0923010F00C9404
:101D7C001F059093240150912001507F992331F03D
:101D8C00503BA9F3503C99F3503E89F3503829F459
:101D9C0088278093220150E909C0503959F426FF55
:101DAC0010C080912201882309F46FC0823048F45E
:101DBC0088270DC0503B09F40EC0503C09F464C098
:101DCC0008C080912201880F8E3F09F48FEF60D0FC
:101DDC005CC086D05AC090912101992311F40C94C7
:101DEC001F05933010F489D050C0973011F0983003
:101DFC0011F49AD04AC0903131F444273091220129
:101E0C000E94290742C0923111F4D8D03EC09331C0
:101E1C0011F4D9D03AC0953211F490D036C0983222
:101E2C00A8F111F4B5D031C0903480F129F430917F
:101E3C002201330F0C94B706913429F4309122010E
:101E4C00330F0C94C006923429F430912201330FD5
:101E5C000C94CB069035D0F0943520F49235B0F438
:101E6C0021D013C0983510F432D00FC0903611F435
:101E7C0095D00BC0903711F49AD007C0973731F436
:101E8C009091220190932101A3D008950C941F05E9
:101E9C0040912401309121010ED080932A010E949F
:101EAC00C80D0895409121013091220140554230D6
:101EBC0010F00C941F05932F942B19F441E0332749
:101ECC0004C03F77469508F430680C94B10D90919E
:101EDC00210191FD0E94B90B882790FD806402C0FE
:101EEC008091210190912201990F803408F091602A
:101EFC0090932A010E94C80D089580912101309180
:101F0C002201823051F0813069F499273A3018F06F
:101F1C003A509395FBCF0C947A0833279091220179
:101F2C000C947A080C941F053091220190FF3C59B7
:101F3C00393C10F40C94D8060C941F0530912201F6
:101F4C00332309F430E880EF0E947B038DE70E9475
:101F5C007B0383E70E947B039091260180912501EE
:101F6C000E94A30986E70E947B03F5E0E09125011E
:101F7C00EA9581910E949209E03031F03A9521F076
:101F8C008CE20E947B03F5CF87EF0E947B030895C0
:101F9C004427309122010E94840608953091220139
:101FAC003A3518F444270C942F0C0C941F053091DF
:101FBC0022013A35D0F744270C94F20B4427309188
:101FCC0022010C9413074427309122010C9406072C
:101FDC0090912401992309F03EC0909121019130F8
:101FEC0019F40E946C3F36C0983019F40E94E20B31
:101FFC0031C0993019F40E94CD0B2CC0903121F4D2
:10200C0078940E942E0726C0953229F40F930E94D3
:10201C0033100F911FC0983711F42F7B1BC09937C9
:10202C0011F4206417C09F37B1F40E94A10AEEF797
:10203C000E94A10AEEF7592F507F0E94A10AEEF7D9
:10204C00692F0E94A10AEEF7503C29F46F3719F45E
:10205C000E94B40C08950C941F050F921F920F93BD
:10206C0080EF0E947B038DE70E947B0383E40E9438
:10207C007B0388E40E947B038DE30E947B038091A9
:10208C0025019091260159D980E20E947B03F091A1
:10209C002801E0912701FE5F508186E40E947B03BA
:1020AC0089E60E947B038EE60E947B038DE30E94EF
:1020BC007B03852F0E94920980E20E947B03F091A2
:1020CC002801E09127016E2F51915F9384E50E94C6
:1020DC007B0388E50E947B038DE30E947B03852FA5
:1020EC001BD980E20E947B0382E50E947B038DE377
:1020FC000E947B035F91852F90912F01903841F0C6
:10210C00899F812D803810F08FEF02C0000C881F42
:10211C0003D980E20E947B036E3F91F187E40E9419
:10212C007B038DE30E947B03819190912F0190386A
:10213C0041F0899F812D803810F08FEF02C0000C88
:10214C00881F0E94920980E20E947B036F3FC1F0BE
:10215C0082E40E947B038DE30E947B03808190913B
:10216C002F01903841F0899F812D803810F08FEF2E
:10217C0002C0000C881F0E94920980E20E947B031F
:10218C008DE40E947B0386E40E947B038DE30E9416
:10219C007B030F7B8091300132D985E20E947B0357
:1021AC0080E20E947B0383E40E947B0383E50E9410
:1021BC007B038DE30E947B0380913A0120D98FE24F
:1021CC000E947B0380913B011AD98FE20E947B0312
:1021DC0080913D018F770E94050A80E20E947B036B
:1021EC0084E50E947B038DE30E947B0380912B018D
:1021FC000E94050A8EE20E947B0380912C01805D77
:10220C000E947B0387EF0E947B030F911F900F901E
:10221C00089512011001020000080E0100000001D7
:10222C00090243000201008031090400000102028E
:10223C0000000524001001052401030004240207FA
:10224C000524060001070583031000400904010062
:10225C00020A000000070581024000010705020286
:10226C004000010009024300020100803109040012
:10227C0000010202000005240010010524010300E6
:10228C0004240207052406000107058303100040FF
:10229C0009040100020A0000000705810240004009
:1022AC00070502024000000A120355006E002000D0
:1022BC004B006E006F0077006E001C03550053003E
:1022CC0042002D00530069006D0070006C00650029
:1022DC0044006D00780000C20100000008000000FE
:1022EC0012010002010000080E01000100010902A8
:1022FC0065000201008031090400000001010000AA
:10230C000924010001090001010904010002010373
:10231C00000007240100014100062402010100060F
:10232C002402020200092403010301020100092412
:10233C0003020401010100090581024000000000B4
:10234C0005250101030905020240000000000525D6
:04235C00010101007A
:0223FE000000DD
:10780000FFFFFF00FFFFFFFFFFFFFFFFFFFFFFFF87
:06781000FFFFFF5060FFC6
:10790000FFFFFF4040FFFFFFFFFFFFFFFFFFFFFF05
:06791000FFFFFF00FFFF76
:107A0000FFFFFFFF00FFFFFFFFFFFFFFFFFFFFFF85
:067A1000FFFF4040FFFFF4
:107B0000FFFFFFFF5060FFFFFFFFFFFFFFFFFFFFD3
:067B1000FFFF00FFFFFF74
:107C0000FFFFFFFFFF00FFFFFFFFFFFFFFFFFFFF83
:067C1000FFFF60FF60FFB2
:107D0000FFFFFF60FF60FFFFFFFFFFFFFFFFFFFFC1
:067D1000FFFFFFFF00FF72
:107E00000C9402035F938F939F93EF93FF93F4324D
:107E100020F4FE3710F00C941F05F999FECF9091D5
:107E200037019B3511F00C941F059927909337016A
:107E3000F89493E00E94423F91E10E94423F80E427
:107E40000D901D900094109491E00E94423F329654
:107E50008A95B1F7FF91EF91EF93FF9395E00E9420
:107E6000423F91E10E94423F87B786FF04C091E103
:107E70000E94423FF9CF7894FF91EF919F918F91AB
:107E80005F91089557B750FDFDCF97BFE8950895CE
:107E90000F7B0895006408950E940C097EF4F09110
:107EA0002801E0912701FE5F9081930F08F49FEF76
:107EB000092E90932A01F2500E94CE0D08950E943F
:107EC0000C09E6F7F0912801E0912701FE5F90810F
:107ED000931B70F79927ECCFE0E0F5E0A0E0B7E066
:107EE00091919D93F630E1F71B7F08950D73696DB5
:107EF000706C65205553422F444D5820496E74656F
:107F0000726661636520666F722041726475696E86
:107F10006F204C656F6E6172646F202876312E3150
:107F20003429000020286329323031352D323120A8
:107F3000572E536368656D6D6572740D00004A7548
:107F40006D706572204F46463A41534349495F631D
:107F50006D64536574202B204D696E69444D582C17
:107F600032353663680D4A756D706572204F4E3A32
:107F70004D4944495F636D645365742C32353663F3
:107F8000680D00004A756D706572204F46463A4193
:107F9000534349495F636D64536574202B204D69D9
:107FA0006E69444D582C32353663680D4A756D70D4
:107FB0006572204F4E3A6F6E6C79204D696E694440
:107FC0004D58206275742035313263680D004D497B
:107FD000444920636828312D3136290020526570CC
:107FE0006561742000005649443D0000205049441A
:027FF0003D0052
:00000001FF
